:100000000C9490000C94B91C0C94921C0C94AD00B0
:100010000C94AD000C94AD000C94AD000C94AD00AC
:100020000C94AD000C94AD000C94AD000C94AD009C
:100030000C94AD000C94AD000C94AD000C94AD008C
:100040000C94481C0C94AD000C94AD000C94AD00C5
:100050000C94AD000C94AD000C94AD000C94AD006C
:100060000C94AD000C94AD000001020304050607DA
:1000700008090A0B0C0D0E0F1011121316150100B2
:100080000100010001000100010001000100010068
:100090000100010001000100010001000100010058
:1000A00001000100010001000100305000000010BB
:1000B0001010101010101010101010101010101040
:1000C000101010101000000000240027002A00006B
:1000D0000000080002010000030407000000000007
:1000E0000000000000000023002600290001020497
:1000F00008102040800102040810200102040810AA
:100100002000000000250028002B00040404040443
:1001100004040402020202020203030303030300B5
:1001200011241FBECFEFD8E0DEBFCDBF11E0A0E0AD
:10013000B1E0EEE3F9E402C005900D92A63BB107F1
:10014000D9F722E0A6EBB1E001C01D92A831B207B9
:10015000E1F70E946C1D0C949D240C9400008230E9
:10016000F8F4E82FF0E0EE0FFF1FE050FF4F2CED0A
:1001700031E031832083813041F0809169008C7FB0
:10018000682B60936900E89A089580916900837FE5
:10019000660F771F660F771F682B60936900E99AD7
:1001A0000895089590E0FC01E153FF4F2491FC0174
:1001B000E351FF4F3491FC01E55FFE4FE491EE23E4
:1001C000C9F0222339F0233001F1A8F4213019F1CC
:1001D000223029F1F0E0EE0FFF1FEF5FFE4FA591F7
:1001E000B4918FB7F894EC91611126C030953E23FD
:1001F0003C938FBF08952730A9F02830C9F02430F0
:1002000049F7809180008F7D03C0809180008F77B7
:1002100080938000DFCF84B58F7784BDDBCF84B53A
:100220008F7DFBCF8091B0008F778093B000D2CFCD
:100230008091B0008F7DF9CF3E2BDACFCF93DF9343
:1002400090E0FC01E351FF4F2491855F9E4FFC013C
:1002500084918823C9F090E0880F991FFC01EB532B
:10026000FF4FA591B491FC01EF5FFE4FC591D49172
:1002700061110DC09FB7F8948C91209582238C93C7
:100280008881282328839FBFDF91CF910895623012
:1002900051F49FB7F8943C91822F809583238C93DF
:1002A000E8812E2BEFCF8FB7F894EC912E2B2C9367
:1002B0008FBFEACF1F93CF93DF93182FEB0161E03D
:1002C0000E941E01209739F460E0812FDF91CF91C9
:1002D0001F910C94D200CF3FD10511F461E0F5CF0E
:1002E000E12FF0E0E153FF4FE491E33031F140F4CE
:1002F000E130B1F0E230E1F0C038D1057CF7E4CF75
:10030000E73029F1E83059F1E430B1F7809180000D
:10031000806280938000D0938B00C0938A0004C0D9
:1003200084B5806884BDC7BDDF91CF911F910895CA
:1003300084B5806284BDC8BDF7CF8091800080689D
:1003400080938000D0938900C0938800EDCF809186
:10035000B00080688093B000C093B300E5CF809177
:10036000B00080628093B000C093B400DDCF3FB78F
:10037000F8948091C0019091C101A091C201B09107
:10038000C30126B5A89B05C02F3F19F00196A11DFA
:10039000B11D3FBFBA2FA92F982F8827BC01CD01CF
:1003A000620F711D811D911D42E0660F771F881F2E
:1003B000991F4A95D1F70895FF920F931F93CF93FA
:1003C000DF930E94B7012091B9013091BA01EB018E
:1003D000C21BD30B2091C6013091C701C217D307AE
:1003E00008F45FC04091CA015091CB0141305105E2
:1003F00061F0E091F301F091F40120813091F50179
:1004000023233091C40123134CC07093BA0160932D
:10041000B9010091C8011091C9014230510509F498
:1004200013C14330510509F44EC14130510561F407
:100430008091B801813009F447C0C8F1833009F4D4
:1004400082C0843009F4C9C08091CA019091CB0167
:10045000019739F1C017D10708F06DC18091B6013D
:100460008F5F8093B6018B30E0F081E090E0909355
:10047000CB018093CA0161E070E08091F1010E949C
:10048000AF001092C4011092B80182E590E0909301
:10049000C9018093C80183E290E09093C7018093E3
:1004A000C601DF91CF911F910F91FF900895C01762
:1004B000D10730F481E08093B801C093B701C4CF75
:1004C00084E08093B801C0CFC017D107D0F5109257
:1004D000B8018091B6018F5F8093B6012091B7017A
:1004E0008C2F0C2E000C990B821B910927FD9395E4
:1004F00097FF03C0919581959109499794F21092C5
:10050000CB011092CA0182E990E09093C9018093D7
:10051000C80182E590E09093C7018093C6011092D4
:10052000B601F090C5016F2D70E08091F1010E943D
:10053000AF008091F50193E0F91227C08093C401C8
:1005400083CF83E0BECFC017D10708F51092CB014F
:100550001092CA0182E990E09093C9018093C8018A
:1005600082E590E09093C7018093C6011092B60196
:10057000F090C5016F2D70E08091F1010E94AF00F5
:100580008091F50133E0F316C9F280E0D7CF909166
:10059000C501933009F482E08093C50182E090E0C8
:1005A0009093CB018093CA0182E990E09093C901B6
:1005B0008093C80182E590E09093C7018093C601C3
:1005C0001092D0018091B6018093D1011092CD019B
:1005D0001092CF011092CE01CBCFC017D107A8F453
:1005E0001092CB011092CA0182E990E09093C90168
:1005F0008093C80182E590E09093C7018093C60183
:100600001092B6011092CD018CCF82E090E09093D1
:10061000CB018093CA0182E990E09093C901809355
:10062000C80182E590E09093C7018093C6011092C3
:10063000D0018091B6018093D1011092CD0110922A
:10064000CF011092CE016DCF9091CD019F5F90931D
:10065000CD018091CE01880FC017D107E0F08093C3
:10066000CE01983009F0F6CEE091D001E630A9F441
:100670001092CB011092CA0182E990E09093C901D7
:100680008093C80182E590E09093C7018093C601F2
:100690001092CD01D9CE8160E2CF83E090E09093BB
:1006A000CB018093CA0181E08E0F8093D00190919D
:1006B000CE01F0E0E653FE4F90878091CF0189276D
:1006C0008093CF01C1CEC017D10728F51092CB017E
:1006D0001092CA011092CD0182E990E09093C90175
:1006E0008093C80182E590E09093C7018093C60192
:1006F0008091CF018111B2CE88E0E0EDF1E0A8ED6C
:10070000B1E001900D928A95E1F781E08093CC01F0
:100710001092B60199CE8091D001863009F4A8CF0D
:1007200082E090E09093CB018093CA011092CD01BA
:100730001092CE0189CE1092B601B3CE2FB7F894A5
:100740006091BC017091BD018091BE019091BF018B
:100750002FBF089508950895CF93DF93FC012BEAEE
:10076000629F212D1124269532E1239FC00111247F
:10077000A481B581A80FB91F322F330F230F621B3D
:10078000462F50E0ED0125E0629FC00DD11D1124E0
:100790002B8123FF1EC011962C9111973FEF320F32
:1007A00011963C93222319F0208521502087A481A3
:1007B000B581A80FB91F65E0649F9001659F300D5A
:1007C0001124A20FB31F13962C911397277F139612
:1007D0002C93A481B581A80FB91F25E0249FE001C7
:1007E000259FD00D1124CA0FDB1F2B8124FF1EC0B3
:1007F00012962C9112973FEF320F12963C932223C0
:1008000019F0218521502187A481B581A80FB91F36
:1008100065E0649F9001659F300D1124A20FB31F06
:1008200013962C9113972F7E13962C93A481B58148
:10083000A80FB91F65E0649F9001659F300D1124DA
:10084000A20FB31F13964C9113974E7F13964C93A0
:10085000A481B581A80FB91FA20FB31F13964C91A5
:1008600013974D7F13964C93A481B581A80FB91FA0
:10087000A20FB31F13964C9113974B7F13964C9373
:10088000A481B581A80FB91FA20FB31F16961C92A1
:1008900044815581480F591F240F351FD9011796E0
:1008A0001C920480F581E02DE80FF91F80818160A2
:1008B0008083DF91CF9108952F923F924F925F9264
:1008C0006F927F928F929F92AF92BF92CF92DF9260
:1008D000EF92FF920F931F93CF93DF93CDB7DEB7C5
:1008E0002B970FB6F894DEBF0FBECDBF9B878A87CC
:1008F000DC0112968C918F3F09F412C180E0F2E185
:100900002F2EA3E03A2EEA85FB859381891708F004
:1009100082C0282F30E0829D80011124E480F58080
:10092000E00EF11ED7019C9190FF5EC0A681B781B9
:1009300012964D915C9113972417350708F054C017
:10094000F7019781448550E070E060E0762F652FD5
:10095000542F4427692B9189492B4B01AA24BB248E
:10096000452E562E672E7724E42CF42E18969C9153
:100970001897992391F0C92ED12CC89C7001C99C5D
:10098000F00CD89CF00C11248F2C949D2001112484
:10099000E52C949FA0011124F52E1E964C911E97D4
:1009A00019966D917C911A971B969C911B974913F0
:1009B00026C09B01839D200D311D11241B964C9157
:1009C0001B97420F532F511DFA0180821C964C91A8
:1009D0001C97420F532F511DFA01E0821D969C91E6
:1009E000290F311DD901FC92EA85FB85A481B581CF
:1009F000A00FB11F9C919E7F9C938F5F84CF220F8D
:100A0000331F220F331F260F371F420F532F511D45
:100A1000FA011082D3CFEA85FB8506811781D801C0
:100A200019968D919C91892B09F47AC0F801C7849D
:100A3000D088E188F2880E94B7016C157D058E058B
:100A40009F0548F40E94B701D8011F966D937D93CE
:100A50008D939C9352970E94B701F801C784D08868
:100A6000E188F2886C197D098E099F096C3271400A
:100A700081059105D8F2F894D80114968D919C9136
:100A800015979A8389831996ED91FC917F01BFEFA9
:100A9000EB1AFB0A80818987F80190810388F48929
:100AA000E02DD80155968C91992309F452C090817C
:100AB000982B98879081809589238F838F818C8351
:100AC00088E08B8358856F8149853B812C818981A2
:100AD0009A81D701508347FD252F3A952083262FF1
:100AE00039F0441F00C000006083000000C0F2CF56
:100AF00038E04D9160830000019761F7D80154966A
:100B0000FC93EE93539749873B832C839A83898385
:100B100078940E94B701F8016787708B818B928B64
:100B20002B960FB6F894DEBF0FBECDBFDF91CF91ED
:100B30001F910F91FF90EF90DF90CF90BF90AF90FB
:100B40009F908F907F906F905F904F903F902F90ED
:100B500008959081982B98879081809589238F8321
:100B60008F818E8388E08D8358856F8149853D8193
:100B70002E8189819A81D701508347FD252F00C09E
:100B800000C0208300C000C000C000C000C060835F
:100B90000000262F3A9541F0441F000000C000C01D
:100BA00000C000C000C0E8CF38E04D9100C06083B5
:100BB00000C0019709F7D8015496FC93EE93539720
:100BC00049873D832E83A2CFDC012BEA629F212D32
:100BD00011242695822F880F820F681B4031A9F0BF
:100BE000403319F1413081F41496ED91FC9182E18A
:100BF000289FE00DF11D112485E0689FE00DF11D97
:100C0000112483818160838308951496ED91FC9172
:100C100082E1289FE00DF11D112485E0689FE00D21
:100C2000F11D112483818260EECF82E1289F900123
:100C300011241496ED91FC911597E20FF31F85E0B6
:100C4000689FB0011124E60FF71F838182608383C0
:100C50001496ED91FC91E20FF31FE60FF71F8381CD
:100C60008460D1CFDF92EF92FF920F931F93CF93C7
:100C7000DF93EC018E81882309F449C0F12C96E0C2
:100C8000E92E0FEF10E08A81F81608F040C0FE9CB4
:100C9000C0011124EB81FC81E80FF91F208120FFA6
:100CA00028C021FF26C023812F5F2383EB81FC8195
:100CB000273008F5E80FF91FA381B0E0A25CBE4F12
:100CC0002C913281239F202D11242583EB81FC81DF
:100CD000E80FF91F658128E0629FB001112481812E
:100CE0009D8190FF04C09801261B370BB9010E941B
:100CF0005A01F394C8CF2E81222311F021502E8364
:100D0000E80FF91F20812D7F20832481DECF8F8182
:100D1000882309F44DC0F12C86E0E82E0FEF10E097
:100D2000DD24DA948A81F81608F042C0FE9CC001E6
:100D30001124EB81FC81E80FF91F208120FF28C0DE
:100D400022FF26C0238121502383EB81FC812223B3
:100D500009F1E80FF91FA381B0E0A25CBE4F2C910E
:100D60003281239F202D11242583EB81FC81E80F04
:100D7000F91F658138E0639FB001112481819D8155
:100D800090FF04C09801261B370BB9010E945A013D
:100D9000F394C8CF2F81211108C0DF82E80FF91F1B
:100DA00020812B7F20832481DFCF22502F83F6CF19
:100DB000DF91CF911F910F91FF90EF90DF900895F9
:100DC000DC0112967C91129730E020E090E07917D8
:100DD000E1F11396ED91FC911497E20FF31F8181DD
:100DE000A9014A5F5F4F86132DC0908190FF25C0F7
:100DF00091FF0AC016969C911697915016969C9357
:100E0000169790819D7F9083908192FF0AC01796DC
:100E10009C911797915017969C93179790819B7F61
:100E2000908390819E7F9083148213964D915C9164
:100E30001497240F351FF901158215966C91617076
:100E40000C94D2009F5F9A01C2CF0895CF93DF9395
:100E5000FC01862F5281D0E0C0E090E0591791F15B
:100E6000A381B481AC0FBD1F11963C911197BE01B7
:100E70006A5F7F4F381365C09C9190FF42C0442346
:100E800031F18FEF820F8F3100F5822F880F880F9D
:100E9000880F14968C93A381B481AC0FBD1F8C91E5
:100EA00081FD03C086818F5F86838C9182608C93E5
:100EB000211101C020E212962C9383819481C80FE6
:100EC000D91F1B82DF91CF9108958FEFE2CF91FF61
:100ED00006C08681815086838C918D7F8C938C9106
:100EE00082FD03C087818F5F87838C9184608C93A0
:100EF00014961C9283819481C80FD91F87E08B833D
:100F0000E1CF6581962F91705FEF520F5F3190F4C2
:100F1000442381F038E0239FB0011124992331F05C
:100F20002FEF30E0A901461B570BBA01DF91CF919B
:100F30000C945A01642F6927832FDF91CF910C9471
:100F4000D2009F5FEB018ACF0F931F93CF938C0149
:100F5000C62FDC0112969C9130E020E080E09817CB
:100F600061F0D8011396ED91FC91E20FF31F2A5F17
:100F70003F4F41814F3F71F4C18361E08C2F0E944C
:100F80001E01F801658161708C2FCF911F910F9127
:100F90000C94D2008F5FE3CFDC0112968C911297F4
:100FA00030E020E090E0891799F01396ED91FC91E4
:100FB0001497E20FF31F2A5F3F4F5181561306C06B
:100FC000413031F480818160808308959F5FEBCF51
:100FD000089508950895DC0113964C91139750E0FD
:100FE00030E020E0241735079CF4C901880F991FD1
:100FF0001496ED91FC911597E80FF91F0190F0817F
:10100000E02D9681947F9B7F96832F5F3F4FEACFA1
:1010100008952F923F924F925F926F927F928F929C
:101020009F92AF92BF92CF92DF92EF92FF920F9377
:101030001F93CF93DF9300D000D0CDB7DEB7213020
:10104000310509F03FC0DC011496CC90B0E0A0E07F
:10105000F3E0BF2EAA24A394AC15A0F5FC01828076
:1010600093808A0E9B1EF4011081FB01868097807D
:101070001B9D800C911C1124F401128112FBDD24B4
:10108000D0F8DA24D016A1F080809180F401D680C7
:10109000D1FA662460F8011103C0D0FA662460F822
:1010A000712C672829F04130510521F410FF07C049
:1010B0001196D2CF41155105D9F711FDF9CF30E086
:1010C00020E0F6CFDC0115962C904090060250905F
:1010D0000702C090FC01D090FD011C821B82EDE054
:1010E0003E2EBB81B21508F08BC0DC01ED91FC9166
:1010F000AB81BC81EA0FFB1F1081DB011896ED91DB
:10110000FC91139DE00DF11D11241485211531056D
:10111000A1F0A081B181109781F010FF0EC016964A
:10112000AC91A1FBEE24E0F8011103C0A0FBEE247A
:10113000E0F8F12CEF2809F45DC012FBAA27A0F912
:10114000B1E0AB27A01709F455C0728441305105B6
:1011500011F411FD4DC0172D7384A12FB0E0AA0F1B
:10116000BB1FAE0FBF1F171508F044C01296EC91BD
:101170001297EF3FD1F1F0E04F01880C991CF2017A
:10118000A384B484F401EA0DFB1DA080B180139602
:101190009C901397E0E26E2E992071F0F60180800A
:1011A000612C891448F09A94998281809280F4018C
:1011B0006980E60DF11D6080992493942115310515
:1011C00009F4912CF501F181FA83F2FB882480F86F
:1011D00098288F2E90FA82F8F50181822115310529
:1011E00021F09380961408F463821F5F1296BBCFA0
:1011F00010E0B3CFAB81BC811196BC83AB8371CFC0
:101200000F900F900F900F90DF91CF911F910F9142
:10121000FF90EF90DF90CF90BF90AF909F908F9016
:101220007F906F905F904F903F902F9008958F9296
:101230009F92AF92BF92CF92DF92EF92FF920F9365
:101240001F93CF93DF93E0900A02F0900B02E0919E
:101250000802F091090280809180D0E0C0E0D701BF
:1012600013968C9113978C171D0639F134F114964F
:10127000ED91FC91CE01880F991FE80FF91FA08016
:10128000B180F501268122FF08C0217000E030E026
:10129000A401B701C5010E940908D50116962C9139
:1012A00023FF09C02695217001E030E0A401B701B9
:1012B000C5010E9409082196D2CF00910602109123
:1012C0000702F12CE12CF8018285F816E8F58F2D44
:1012D00090E0880F991F0384F485E02DE80FF91F33
:1012E000C081D181898182FB442740F92B81869579
:1012F0008170481303C08A81821721F1898140FBE4
:1013000081F989832A83E0910602F091070280FB2C
:10131000CC24C0F8D12CC601880F991FE80FF91F03
:1013200081819281DC01ED91FC910480F581E02DB9
:101330006881099581E099819B7F99831B82E82AC6
:10134000F394C1CF80E0F7CFEE20B1F0C0E0F80118
:101350008081C81788F4EC2FF0E0EE0FFF1FE00F3C
:10136000F11F81819281DC01ED91FC910680F78172
:10137000E02D0995CF5FEBCFDF91CF911F910F91BA
:10138000FF90EF90DF90CF90BF90AF909F908F90A5
:101390000895CF93C82F80E090E0892B51F0809181
:1013A000E2018C1731F081E0C11101C080E00E94A0
:1013B0000000C093E20160E070E0CB01C1110E9427
:1013C0009E036093E3017093E4018093E5019093A1
:1013D000E60180E090E0892B59F08091E2018C17C2
:1013E00039F081E0C11101C080E0CF910C94000080
:1013F000CF910895642FA091FA01B091FB0141E0D3
:1014000050E02130310511F050E040E0ED91FC91C9
:1014100011970084F185E02D262FBC01CD010994A0
:10142000A091FA01B091FB01ED91FC91119706801A
:10143000F781E02DBC01CD010994462FA091FA015E
:10144000B091FB01ED91FC9111970480F581E02DA5
:10145000BC01CD0109940895A091FA01B091FB015E
:10146000ED91FC9111970280F381E02DBC01CD013B
:101470000994A091FA01B091FB0141E0611101C012
:1014800040E0ED91FC9111970190F081E02DBC01BD
:10149000CD0109940C94390A80E090E0892B29F061
:1014A0008091F90183FD0C9400000895CF93DF93A0
:1014B000EC0161E08B810E94D20081E089870E946B
:1014C0009E036A5F7F4F8F4F9F4F6D837E838F8315
:1014D000988783E08C83DF91CF9108958091FA0102
:1014E0009091FB010C94560A0C946E0ACF92DF92F5
:1014F000EF92FF92CF93DF93EC01888180FF14C0BD
:10150000C980DA80EB80FC800E949E03C61AD70A4D
:10151000E80AF90A9EEF1C141D041E041F040CF4B3
:101520009FEF88818923888388818170DF91CF91A3
:10153000FF90EF90DF90CF9008950F93CB01642F31
:10154000422F202FDC01ED91FC910280F381E02DF0
:101550000F910994CB01642FDC01ED91FC91019076
:10156000F081E02D422F0994CF93DF93FC01EA0133
:101570008089861799F0608B8FEF9FEF928B818B1C
:10158000138A662359F0683208F052C0613069F45A
:1015900081E1838B81E090E0928B818B83898883CA
:1015A00081899289DF91CF910895613121F4638B14
:1015B00081E190E0F1CF623129F481E1838B82E116
:1015C00090E0EACF673039F486E1838B87E090E0E2
:1015D000222311F3E3CF683039F487E1838B88E06D
:1015E00090E02223C9F2DACF6D3129F489E1838BAF
:1015F0008DE190E0D1CF6E3129F489E1838B8EE1CA
:1016000090E0CACF6F3129F489E1838B8FE190E0BC
:10161000C3CF603229F489E1838B80E290E0BCCFB4
:10162000613209F0BBCF89E1838B81E290E0B4CFD6
:1016300028ED260F283408F580E2838B822F66E0A0
:101640000E942523382F822F90E066E070E00E94F0
:1016500031232085321708F0A1CF23E2009729F02B
:1016600024E28130910509F025E2238B26E0329FA8
:10167000800D911D112488968FCF80E9860F8530CB
:1016800060F490E4938B9285891708F087CF97E4F4
:10169000938B90E080599F4F7FCF65578485681763
:1016A00008F07CCF89E5838B70E06B587F4F728B9D
:1016B000618B74CF089508950895CF93DC015096FF
:1016C000ED91FC913097D9F0E617F707F1F4C22FAE
:1016D000E0910802F0910902808191818427952789
:1016E000019721F4518340830E941709E091080279
:1016F000F09109028481C81741F0C48306C0FC013F
:10170000868597858617970711F3CF910895CF9215
:10171000DF92EF92FF920F931F93CF93DF934130AD
:10172000510519F4220F25FD2160DC011E96ED9173
:10173000FC911F97E617F70791F050968D919C91B9
:10174000009721F011E08617970751F0DF91CF91B4
:101750001F910F91FF90EF90DF90CF90089510E0D0
:101760008FEF840F853090F75527FA01E85CFE4F24
:10177000DF0111974C91F080C0910A02D0910B02C9
:10178000B0E0A0E050E030E04F1508F042C0C901E1
:101790000A2E02C0959587950A94E2F7982F9170CA
:1017A0006C85862F817060FD812FEB8070E060E09A
:1017B0006E1528F080E0582B4F5F1196E5CF6B0136
:1017C000CC0CDD1CEC81FD81EC0DFD1D0190F08148
:1017D000E02D07816F5F7F4F041750F34013EACF6E
:1017E00081110CC0868184608683682F617090FBB4
:1017F00080F96917F9F2868381E0DDCF8681886000
:10180000868381FB662760F96917A1F290FB81F955
:10181000F2CF552309F49ACFDF91CF911F910F9109
:10182000FF90EF90DF90CF900C9417090F931F93C8
:10183000CF93DF931F92CDB7DEB70091FE011091D9
:10184000FF01D801ED91FC910190F081E02D20E0A5
:10185000AE014F5F5F4FC80109958F3F980781F038
:10186000D801ED91FC910680F781E02D4981BC0102
:10187000C80109950F90DF91CF911F910F910895A5
:1018800080E0F8CFCF93DF931F92CDB7DEB7242F40
:101890008091FE019091FF01DC01ED91FC9101909E
:1018A000F081E02DAE014F5F5F4F099521E0019679
:1018B00009F420E0822F0F90DF91CF910895E42F5B
:1018C000F0E0E155FF4F84910895E42FF0E0E655F4
:1018D000FF4F84910895D90186E0483038F5E42F10
:1018E000F0E0EB58F34F0C9459237D0C840C870CDB
:1018F0008A0C960C8D0C900C930CEEE0F1E00190AC
:101900000D928A95E1F70895E4E1F1E0F8CFEAE17C
:10191000F1E0F5CFE0E2F1E0F2CFE6E2F1E0EFCF87
:10192000ECE2F1E0ECCFE2E3F1E0E9CFFD0111926E
:101930008A95E9F7089586ED96E008958AED96E098
:101940000895E62FF0E0EE0FFF1FE258FF4F84915D
:1019500090E00895E62FF0E0E859FF4F8491089554
:1019600086E108957F928F929F92AF92BF92CF921D
:10197000DF92EF92FF920F931F93CF93DF93DC01DF
:1019800013961C9113971496ED90FC90159790E088
:1019900080E0782E5C01AA0CBB1CAE0CBF1CE501DC
:1019A000E881F981811720F401962781261788F3B1
:1019B000309719F087818617E9F112968C9112976A
:1019C0008117C0F1062F6D01E12FF0E0EE0FFF1F30
:1019D000EE0EFF1EF701C081D1812097B1F488E09F
:1019E00090E00E945F23EC01F60180801C821D8242
:1019F0008FEF8F83912CC4010E945F239B838A8386
:101A0000C4010E945F23998388830F838E81847F22
:101A10008B7F8E8381E0810FF6018383F70171163E
:101A200030F492918291938382831150F8CFF50123
:101A3000D183C083872DDF91CF911F910F91FF90AC
:101A4000EF90DF90CF90BF90AF909F908F907F905E
:101A500008950E94C909E0EEF1E081E087831086D5
:101A6000E9EEF1E088E0DF011D928A95E9F708953B
:101A70002F923F924F925F926F927F928F929F929E
:101A8000AF92BF92CF92DF92EF92FF920F931F938C
:101A9000CF93DF9300D000D0CDB7DEB79C838B838C
:101AA000DC0118968C91B12C882309F45EC1E12CDD
:101AB00035E0F32E42E3442E512C612C712C54E17D
:101AC000352EEB81FC818381E81608F04EC1F2E1EE
:101AD000EF9E80011124AB81BC811496ED91FC91A5
:101AE000E00FF11F8181882309F44EC090E080E06F
:101AF000EB81FC8124813581200F311FF89ED001BC
:101B0000F99EB00D1124F901EA0FFB1F7381AC019E
:101B10004F5F5F4F6A0170FF63C073FB662760F918
:101B200073FF5EC025812F5F2583EB81FC8144819B
:101B30005581FA01E00FF11F273040F5AE0FBF1FAE
:101B4000FC9CC001FD9C900D1124E80FF91FE08161
:101B5000F0E0E25CFE4F808114969C911497899F7F
:101B6000802D112417968C93AB81BC811496ED9136
:101B7000FC91E00FF11F808181608083B62EC60149
:101B80008330910509F0B4CFE3949BCF21813FEFDF
:101B9000320F3183222341F0AB81BC8118962C9106
:101BA0001897215018962C93AB81BC811496ED9117
:101BB000FC911597E00FF11FF89E9001F99E300DF2
:101BC0001124E20FF31F8381877F83831496ED91A5
:101BD000FC91E00FF11FE20FF31F86818783C4CFD2
:101BE000F89ED001F99EB00D1124F901EA0FFB1FF8
:101BF000238121FFC4CF23FB222420F823FFBFCF62
:101C000045814F5F4583EB81FC8124813581F9015A
:101C1000E00FF11F5D01AE0EBF1ED50114962C9191
:101C20006B817C81AAE2A29F600D711D11249B0132
:101C3000DB011F965C915417D8F0FC9CC001FD9C01
:101C4000900D1124E80FF91F8081280F311DF90133
:101C50008785D50117968C93AB81BC811496ED9145
:101C6000FC91E00FF11F808181608083B22C87CFCF
:101C700021813FEF320F3183222329F0EB81FC8158
:101C8000208521502087EB81FC81A481B581A00FA4
:101C9000B11FF89EF001F99EF00D1124AE0FBF1F89
:101CA00013962C911397277F13962C93AB81BC81AD
:101CB00014962D913C91D901A00FB11FEA0FFB1F83
:101CC000238122FF4FC012962C91129731E0320FE0
:101CD00012963C93211105C0EB81FC8121852F5F79
:101CE0002187AB81BC811496ED91FC91E00FF11F2F
:101CF000F89E5001F99EB00C1124EA0DFB1D838162
:101D0000806183830E945422EB81FC812481358190
:101D1000200F311F49018A0C9B1CA30192010E94D4
:101D2000C222625E7F4F8F4F9F4FD40114966C93F7
:101D3000AB81BC811496ED91FC911597E00FF11FDA
:101D4000FC9CC001FD9C900D1124E80FF91F10822E
:101D500014968D919C91800F911FA80EB91EF501CC
:101D600037827ACF8681878377CFEB81FC8181852B
:101D7000882309F422C11982E12C85E0F82E9AE526
:101D8000492E512C612C712C24E1A22E3324339442
:101D9000AB81BC8113968C91E81608F00CC1B2E1BE
:101DA000EB9E80011124AB81BC811496ED91FC91D6
:101DB000E00FF11F8281882309F44FC030E020E05A
:101DC000EB81FC8184819581800F911FF29EA0019F
:101DD000F39E500D1124FC01E40FF51FA381B901FE
:101DE0006F5F7F4F4B01A0FF61C0A4FB662760F9C6
:101DF000A4FF5CC0858181508583AB81BC81149632
:101E0000ED91FC91E00FF11F882349F1DF01A40F50
:101E1000B51FF89CC001F99C900D1124E80FF91F23
:101E2000E081F0E0E25CFE4F808114969C91149773
:101E3000899F802D112417968C93AB81BC811496B9
:101E4000ED91FC91E00FF11F8081816080836983B7
:101E500094012330310509F0B3CFE39499CF828107
:101E60009FEF980F9283882329F0EB81FC81818575
:101E700081508187AB81BC811496ED91FC911597BF
:101E8000E00FF11FF29EC001F39E900D1124E80FA8
:101E9000F91F23812F7E23831496ED91FC91E00F8F
:101EA000F11FE80FF91F86818783C7CFF29E60017B
:101EB000F39ED00C1124FC01EC0DFD1D838181FFEC
:101EC000C7CF84FB222420F884FFC2CF85818F5F97
:101ED0008583AB81BC811496ED91FC91E00FF11FDD
:101EE000EC0DFD1D94818913B3CF8781843181F579
:101EF0000E945422AB81BC811496ED91FC91159700
:101F0000E00FF11FEC0DFD1D34821496ED91FC9154
:101F10001597E00FF11FF89CC001F99C900D11245A
:101F2000E80FF91F10821496ED91FC91E00FF11F5C
:101F3000EC0DFD1D86818783AB81BC811496ED91EC
:101F4000FC91E00FF11F808181608083298280CF26
:101F50000E945422EB81FC8124813581200F311FA6
:101F6000A9014C0D5D1D5A834983A30192010E9472
:101F7000C222625E7F4F8F4F9F4FA981BA81149614
:101F80006C93AB81BC811496ED91FC911597E00F99
:101F9000F11FF89CC001F99C900D1124E80FF91F66
:101FA000108214968D919C91800F911FC80ED91E9E
:101FB000F601A782C1CFB981BB2ABB2001F1AB8159
:101FC000BC81ED91FC9111970680F781E02DCD0148
:101FD0000F900F900F900F90DF91CF911F910F9165
:101FE000FF90EF90DF90CF90BF90AF909F908F9039
:101FF0007F906F905F904F903F902F9009940F903B
:102000000F900F900F90DF91CF911F910F91FF9044
:10201000EF90DF90CF90BF90AF909F908F907F9088
:102020006F905F904F903F902F9008954F925F92E6
:102030006F927F929F92AF92BF92CF92DF92EF9278
:10204000FF920F931F93CF93DF93EC018BEA689F6E
:10205000812D1124869592E1899F70011124EC81D4
:10206000FD81EE0DFF1D982F990F890F681B062F1C
:1020700010E0442309F4B5C08FEF820F8F3108F0D0
:102080005EC0822F880F880F880F95E0909FD00147
:10209000919FB00D1124EA0FFB1F8683EC81FD8117
:1020A000EE0DFF1DAE0FBF1F13968C91139780FF8F
:1020B00048C0818191E0980F9183811103C0888588
:1020C0008F5F8887EC81FD81EE0DFF1D35E0309F2D
:1020D000C001319F900D1124E80FF91F83818860A2
:1020E0008383211101C020E2EC81FD81EE0DFF1DF3
:1020F00085E0809FA001819F500D1124E40FF51F02
:102100002483EC81FD81EE0EFF1E0F5F1F4F809F29
:10211000F001819FF00D1124EE0DFF1D1082DF9163
:10212000CF911F910F91FF90EF90DF90CF90BF90D4
:10213000AF909F907F906F905F904F9008958FEF3A
:10214000A4CF81FF42C0818191E0980F91838111DA
:1021500003C088858F5F8887EC81FD81EE0DFF1DB0
:1021600085E0982E909E5001919EB00C1124EA0DAE
:10217000FB1D8381886083830E945422CC80DD8094
:10218000CE0CDF1CCA0CDB1C22E0422E512C612C31
:10219000712CA30192010E94C222F60164830E9465
:1021A00054220C80DD81C02DEC0EFD1E0F5F1F4FF1
:1021B000909EE001919ED00D1124CE0DDF1DA30154
:1021C00092010E94C2226883AACF16968C9116971C
:1021D00017968C93EC81FD81EE0DFF1D808181604F
:1021E00061C085E0809FD001819FB00D1124AE0FAA
:1021F000BF1F13968C9183FF18C081819FEF980FAA
:102200009183882319F0888581508887EC81FD812E
:10221000EE0DFF1D25E0209FC001219F900D112490
:10222000E80FF91F8381877F8383EC81FD81EE0DA9
:10223000FF1D85E0809FD001819FB00D1124AE0F5E
:10224000BF1F13968C9180FF2FC0828191E0980F61
:102250009283811103C089858F5F8987EC81FD811D
:10226000EE0DFF1D85E0809F9001819F300D1124B0
:10227000E20FF31F938190619383EC81FD81EE0D5A
:10228000FF1DE20FF31F1682EC81FD81EE0EFF1E93
:102290000F5F1F4F809FF001819FF00D1124EE0D05
:1022A000FF1D87E080833BCF84FF18C082819FEFB2
:1022B000980F9283882319F0898581508987EC8152
:1022C000FD81EE0DFF1D25E0209FC001219F900D97
:1022D0001124E80FF91F83818F7E8383AC81BD8138
:1022E000AE0DBF1D25E0209FC001219F900D112440
:1022F000A80FB91F16961C92EC81FD81EE0DFF1DF3
:10230000E80FF91F178266CF0E9484240C942C0AD0
:10231000CF93DF932091F6013091F7012F3F3207E1
:1023200021F0C901DF91CF9108958091F90187FFD4
:102330002BC086FF0FC089E090E00E948611C82F55
:1023400081E090E00E9486119C2F9093F70180938A
:10235000F60115C089E090E00E948611C82F81E047
:1023600090E00E94861190E4C99F90011124207C86
:1023700031708F73282B3093F7012093F6018091F1
:10238000F6019091F701CECF85FF0CC081E190E07E
:102390000E948611C82F82E190E00E948611C05CE5
:1023A000DD0BD2CF81E090E00E94861190E0CDCF8E
:1023B000CF92DF92EF92FF920F931F93CF93DF9311
:1023C000EB017B0120E2E20EF11C8B016C01C61ACD
:1023D000D70AC601800F911F0E94AC22F801819399
:1023E0008F01EE15FF05A9F7CE01DF91CF911F9167
:1023F0000F91FF90EF90DF90CF900895CF92DF92F2
:10240000EF92FF920F931F93CF93DF93EB017B012A
:1024100025E0E20EF11C8B016C01C61AD70AC60139
:10242000800F911F0E94AC22F80181938F01EE155D
:10243000FF05A9F7CE01DF91CF911F910F91FF907A
:10244000EF90DF90CF900895CF92DF92EF92FF92BE
:102450000F931F93CF93DF93EB017B0126E0E20EF6
:10246000F11C8B016C01C61AD70AC601800F911F9F
:102470000E94AC22F80181938F01EE15FF05A9F7A8
:10248000CE01DF91CF911F910F91FF90EF90DF90E0
:10249000CF900895CF92DF92EF92FF920F931F9308
:1024A000CF93DF93EB017B0128E2E20EF11C8B015D
:1024B0006C01C61AD70AC601800F911F0E94AC2278
:1024C000F80181938F01EE15FF05A9F7CE01DF9189
:1024D000CF911F910F91FF90EF90DF90CF900895D3
:1024E0002F923F924F925F926F927F928F929F9224
:1024F000AF92BF92CF92DF92EF92FF920F931F9312
:10250000CF93DF93CDB7DEB7E2970FB6F894DEBF77
:102510000FBECDBF5C01762E8A01BE016F5F7F4F7B
:10252000DC011D968D919C910E944A12872D8F7E11
:1025300009F431C1B0E27B1258C1912C812CD50134
:102540001D968D919C918896BE016F5F7F4F880D7F
:10255000991D0E9424128981682F6F7109F498C116
:10256000E0900A02F0900B0286FB332430F8DD2461
:10257000D394B82FB0724B2E85FDD12C85E0FE018F
:102580003296DE01999601900D928A95E1F75A8074
:10259000F7018181681708F060E0C7010E94B20C62
:1025A000682ED7011B968C911B972C9110E000E0B0
:1025B000821778F591E0980F1B969C931B971896BD
:1025C0000D911C91BDE08B9F000D111D1124F80190
:1025D00011821082D7011D964D915C911E975383F5
:1025E00042831D964D915C911E97558344831D96A1
:1025F0004D915C911E97578346831D964D915C913A
:10260000518740871286138694859C7F9B7F948791
:10261000282EF8018485D0FA81F9848744E0438725
:1026200082E0411080E0D8011A968C93F7018485EE
:10263000982F917080FD932DD8011C968C911C973A
:1026400090FB82F91C968C93652D6F7109F466C01E
:10265000F7018285D12CC12C8217A0F491E0980F4C
:102660009287C680D780F3E08F9FC00CD11C1124C5
:10267000D7011F962D913D914C91F6012083318316
:10268000428388ABD60112968C91129730FA82F968
:1026900012968C931297F801848557FA80F98487F3
:1026A000411009C012968C91129756FA80F955FA8A
:1026B00081F912968C93D70111968C91681708F0C6
:1026C00060E0C7010E94B20CF70124813581E82F38
:1026D000F0E0EE0FFF1FE20FF31FA081B181F801C0
:1026E000B183A083862D90E0880F991F280F391F92
:1026F000F90180819181F6019183808312968D91F9
:102700009C9113971496EC91149721E02E0F149638
:102710002C93E80FF92FF11D48A94083D8011B968F
:10272000DC90E0910602F0910702FAABE9AB2E01D2
:10273000FAE24F0E511CF80170E0D71609F48EC072
:10274000D2016D912D01062F0F7111F1A9A9BAA91E
:102750001A96CC9090E080E0182F8C1508F07CC081
:102760009C01220F331FA9A9BAA91B964D915C9118
:10277000240F351FD9012D913C91D90114962C912C
:1027800001960213E9CF12836295669567706383A1
:102790007F5F3296D2CFBE016F5F7F4FF501858597
:1027A00096850E944A12D8012D913C91EDB7FEB753
:1027B000B8970FB6F894FEBF0FBEEDBFADB7BEB76A
:1027C000119688E2FE01319601900D928A95E1F70B
:1027D000D901ED91FC91C80109950FB6F894DEBFBF
:1027E0000FBECDBF772009F4A8CEF0E47F125DC004
:1027F000D5011D968D919C91BE016F5F7F4F8059D1
:102800009F4F0E94FE11A091FC01B091FD019E011D
:102810002F5F3F4F90E080E050E24C91481719063F
:1028200009F00CF440C0F90141919F011196ED911E
:10283000FC911297E80FF91F4695469546954083FF
:102840001196ED91FC911297E80FF91F408141110B
:1028500001C050830196E1CF10E095CF862D90E026
:10286000880F991FF70124813581820F931FFC0186
:10287000A081B1818D919C9111971596EC9115973E
:1028800021E02E0F15962C93E80FF92FF11D2082D1
:10289000F6E08F0E911C48E48416910409F04FCEA7
:1028A0007110A3CFA5CF772019F0B0E57B1245C0FA
:1028B000D5011D968D919C91BE016F5F7F4F8B5806
:1028C0009F4F0E94D811E0900602F090070210E09E
:1028D000F7018285181788F5212F30E0C901880F8C
:1028E000991F0384F485E02DE80FF91FA081B181C1
:1028F000E0910602F091070211968C911197817078
:102900008EA71FA68EA59FA5880F991FE80FF91FF8
:102910008181928141E050E04C0F5D1F240F351FF3
:10292000FC0140815181FA01C280D380F9014081CC
:102930006C91F60109951F5FCBCFE2960FB6F89424
:10294000DEBF0FBECDBFDF91CF911F910F91FF90E2
:10295000EF90DF90CF90BF90AF909F908F907F903F
:102960006F905F904F903F902F900895CF92DF929D
:10297000EF92FF920F931F93CF93DF938C01C62F9B
:10298000C07FC034D9F480910A0290910B020E945A
:10299000EB07A091FC01B091FD0190E080E02C914B
:1029A0002817190609F00CF475C01196ED91FC91E9
:1029B0001297E80FF91F10820196F1CF607D09F49C
:1029C00042C0C03509F06AC0C0900602D09007022C
:1029D000D0E0D6011A968C911A97D81708F05EC0ED
:1029E0008D2F90E0880F991F1B96ED91FC91E80FB9
:1029F000F91FA081B18111968C91119713961C92A9
:102A000013978B7F8D7F11968C93119712961C9242
:102A10001297E0910602F091070280FBEE24E0F8A5
:102A2000F12CC701880F991FE80FF91F818192814E
:102A3000FC0120813181F901208531856C91F901FA
:102A40000995DF5FC6CFE0910A02F0910B02238166
:102A500030E090E080E04FEF82179307A4F4BC01D0
:102A6000660F771FA481B581A60FB71F0D90BC918B
:102A7000A02D17964C93179714961C9214971596A1
:102A80001C920196E9CF138212861386CC2309F497
:102A900080CF97CFCC2309F497CF93CFA801445F81
:102AA0005F4F6C2F8091FE019091FF01DF91CF91DC
:102AB0001F910F91FF90EF90DF90CF900C947012C8
:102AC000CF93DF93EC018C899D898617970749F096
:102AD0007D8B6C8B8D859E85860F971F0E94AC2207
:102AE0008E8B8E89DF91CF9108958331910588F483
:102AF0008131910530F48130910519F089309105CB
:102B000031F42FEF3FEF3093F7012093F6010C944F
:102B10001D0A8D319105D9F7677F6093F9012091E6
:102B2000E0012F73362F307C232B2093E001E9CF77
:102B3000BF92CF92DF92EF92FF920F931F93CF93AA
:102B4000DF938B01B42E690182FF23C083FF17C07E
:102B500061E0C8010E944A0A8823D9F16B2DC8019F
:102B60000E9475158B1135C0F601DF91CF911F9131
:102B70000F91FF90EF90DF90CF90BF90099460E0AD
:102B8000C8010E944A0A882321F1C8010E948611C7
:102B9000E9CF842F8770C1E0D0E07E0101C0EE0C48
:102BA0008A95EAF7D42FD870CB010E948611C82FDE
:102BB000B4FE1CC061E0C8010E944A0A882349F0A3
:102BC000DD2389F0CE296C2FC8010E9475158C1762
:102BD00059F2DF91CF911F910F91FF90EF90DF900D
:102BE000CF90BF900895E094CE21EDCF60E0C80172
:102BF0000E944A0A882369F3CE21DD2319F0C1110E
:102C0000B3CFE7CFCC2309F4AFCFE3CFCF92DF929E
:102C1000EF92FF920F931F93CF93DF937C016B0191
:102C2000C42F122FD42FD07E8091E00187FF2CC0BB
:102C3000D03EC1F58091E1018823A1F190E00E948E
:102C40008611D82F8091E10190E001960E948611B3
:102C5000982F8D2FE816F90629F56C2F70E0762F46
:102C6000662766277370612B6F5F7F4F2CE43AE015
:102C7000402F8C2FDF91CF911F910F91FF90EF90FC
:102C8000DF90CF900C94981580FD32C0D03609F4B7
:102C900064C088F4D03209F447C0D03409F45DC070
:102CA000DD2379F1DF91CF911F910F91FF90EF908C
:102CB000DF90CF900895D03A09F483C090F42C2F80
:102CC0002F7141E050E0D03869F7B601C701DF91BC
:102CD000CF911F910F91FF90EF90DF90CF900C94C8
:102CE000100AD03C09F476C0D03E09F4B6CFDACF52
:102CF0000E9488118E159F0549F2E114F10431F20A
:102D0000D1CF8C2F8E7071F680E090E0892B51F23C
:102D10008C2F8170DF91CF911F910F91FF90EF90D9
:102D2000DF90CF900C940000CF71CF3109F0BACF73
:102D3000412F4F7771F0413071F0111F1127111F92
:102D4000212F30E00FE710E0B601C7010E94FA0919
:102D5000A9CF41E0F2CF40E0F0CF2C2F30E08C2F14
:102D60008F71813029F030F0803121F08131F9F418
:102D700040E001C041E025FB222720F90DE110E0F1
:102D800030E0B601C7010E94FA0980E090E0892B8B
:102D900009F488CF4C2FB601C701DF91CF911F9165
:102DA0000F91FF90EF90DF90CF900C940000C9013D
:102DB000880F991F8E71C4FB442740F9482B42505D
:102DC000DACF2C2F2F7043E050E0C4FF7ECF42E0DB
:102DD00050E07BCFCF71CE3139F0CF3109F062CFE7
:102DE000212F45E050E071CF212F44E050E06DCF1E
:102DF000FF920F931F93CF93DF93EC01F62E088180
:102E00001981C8010E94AC22F81621F06F2DC8016B
:102E10000E94B422CE01DF91CF911F910F91FF90BC
:102E200008952F923F924F925F926F927F928F926E
:102E30009F92AF92BF92CF92DF92EF92FF920F9349
:102E40001F93CF93DF93CDB7DEB7E4970FB6F89417
:102E5000DEBF0FBECDBF7C01462E542E8E010F5F0C
:102E60001F4FB801DC011D968D919C910E944A1262
:102E70006E01B9E2CB0ED11C460196EFA92E93E06C
:102E8000B92E3601C5010E94AC22F40181934F0195
:102E9000FFEFAF1ABF0AA11484E0B80699F75110EA
:102EA00001C059A4D7011D96AD90BC901E978A8190
:102EB00018166CF589858D3051F58885803139F586
:102EC000411025C0B501695F7F4FED91FC910084F1
:102ED000F185E02D20E040E1C7010995E4960FB6A9
:102EE000F894DEBF0FBECDBFDF91CF911F910F9140
:102EF000FF90EF90DF90CF90BF90AF909F908F901A
:102F00007F906F905F904F903F902F900895A11405
:102F1000B4E0BB0640F460E0C5010E94B422EFEFCC
:102F2000AE1ABE0AF4CF89A5851159A686EFA82E40
:102F300083E0B82EBCAAABAAD6016D916D01CE017B
:102F4000C3960E94F816BFEFAB1ABB0AA114E4E0C7
:102F5000BE0681F788E2D8011D928A95E9F78DE0D7
:102F6000898780E1888782E08E8FF7018789908D3D
:102F7000DC01ED91FC910190F081E02D652D09952A
:102F8000009729F08038910508F08DC08A83F701F9
:102F90008789908DDC01ED91FC910280F381E02D19
:102FA000652D0995009729F08038910508F084C0B7
:102FB00088A3F701C584D6845801C01AD10AC60176
:102FC0008A0D9B1D9CAB8BABD5016D915D01CE0134
:102FD000C3960E94F8166A147B0489F7B12CA12CC1
:102FE000412CF70132963F011801F6E02F0E311CFB
:102FF000D7011D968D919C918896B8018A0D9B1DD5
:103000000E94241286E0F301D80101900D928A9566
:10301000E1F7552079F0F7018789908D009751F0FD
:10302000DC01ED91FC910480F581E02D9801442DA7
:10303000652D0995F701C584D684F8E2CF0ED11C21
:10304000CA0CDB1C4801C01AD10AC601880D991DA3
:103050009CAB8BABD4016D914D01CE01C3960E9408
:10306000F8162814390489F74394B6E0AB0EB11C66
:10307000ECE04E12BDCFD7011D968D919C91B80109
:1030800080599F4F0E94FE11F701828590E0F80160
:103090009F01201B310B28173907ACF4D701199673
:1030A0002C912193F5CF2E8D22622E8F23E02A833F
:1030B00090549A8B8B8B6BCF2F8D21602F8F9054D8
:1030C00099A38AA376CF5520F1F0F7018789908DD7
:1030D000892BC9F0D12CD7011A968C911A97D81642
:1030E00090F457968D919C91DC01ED91FC910680B6
:1030F000F781E02D4D2D652D0995F801ED0DF11DA0
:103100008083D394E8CFF701C584D6844601F0E7E5
:103110008F0E911C85E7C80ED11C58019CAA8BAA62
:10312000D5016D915D01CE01C3960E94F816BFEFE7
:103130008B1A9B0AC814D90489F7F70185859685EF
:10314000B8018B589F4F0E94D811D7011B962C9124
:10315000C80180966801F60121936F018E179F07C1
:10316000D1F75520E1F0D70157968D919C91892B8D
:10317000B1F0B12CF7018485B81688F48789908D59
:10318000DC01ED91FC910084F185E02D4B2D652D46
:103190000995F801EB0DF11D8083B394EBCFF70196
:1031A000E584F684E01AF10AC7018B589F4F7C0131
:1031B000C701800F911F9CAB8BABD8016D918D0126
:1031C000CE01C3960E94F816C016D10689F786CEA6
:1031D000AF92BF92CF92DF92EF92FF920F931F9325
:1031E000CF93DF931F92CDB7DEB77C01C42E009141
:1031F000FE011091FF01D801ED91FC910190F08149
:10320000E02D21E0AE014F5F5F4FC80109955C01E1
:103210000196A1F4D12CF701828181113EC08981F0
:103220008F708630A8F5833010F48130B1F5DD2041
:10323000A1F1C7010E94560A698148C0D801ED91E9
:10324000FC910280F381E02D2C2D4981B701665F4E
:103250007F4FC8010995D82E8823E1F2D801ED915E
:10326000FC910680F781E02D4981B501C8010995DF
:10327000C81661F0D801ED91FC910084F185E02D34
:1032800029814C2DB501C8010995C5CF1982C3CF3D
:10329000873081F010F08B3050F28D2D0F90DF9140
:1032A000CF911F910F91FF90EF90DF90CF90BF9043
:1032B000AF900895C7010E94560A40E061E08091F6
:1032C000FE019091FF010E94111760E0C7010E946A
:1032D000B614E3CFCF93DF9300D0CDB7DEB7FB01B9
:1032E0002F702730B9F0DC0154962D913C91559701
:1032F0006217730711F456964C93642FDC011D96E8
:103300008D919C91E80FF91FFA83E983CE01019614
:103310000E94F8160F900F90DF91CF910895BF9201
:10332000CF92DF92EF92FF920F931F93CF93DF9391
:103330007C018091E2018823B1F00E949E030091FC
:10334000E3011091E4012091E5013091E601601B59
:10335000710B820B930B653171058105910518F096
:1033600080E00E94290D8091CC018823B1F1F8946E
:1033700088E0E8EDF1E0ACE0B2E001900D928A95D2
:10338000E1F71092CC01789480910C02E82FF0E0E4
:10339000E25FFD4F863018F411928F5FFBCF80E023
:1033A00090E0892B21F08CE092E00E940000809157
:1033B0000E0281114AC090910F02911146C080E027
:1033C00090E0892B19F080E00E9400008091E201DA
:1033D0008823B9F181E00E94C909D70119968C911F
:1033E000882371F0C70104960E94760A811108C0F3
:1033F00060E0F70183810E94D200D70119961C92E8
:103400000091060210910702C80105960E94760AF3
:10341000811134C2C0E0F8018081C81708F021C2D0
:10342000EC2FF0E0EE0FFF1FE00FF11F8181928182
:10343000DC01ED91FC910284F385E02D0995CF5FCD
:10344000EACF81E00E94290DC8CF9091E201992333
:1034500009F482C08057803108F07BC081E00E946F
:10346000C909C0910C028091E901C8130AC04C2F10
:1034700050E06BEE71E08EE092E00E948924892B8F
:1034800061F01092E80188E0ECE0F2E0A9EEB1E032
:1034900001900D928A95E1F7A0CF8091E8018F5FAE
:1034A0008093E801C330E9F520910E02822F8770E6
:1034B00010910F02853029F41093E7010E946E0AE3
:1034C0008CCFCDE1D0E0843089F0C82FD0E08430BB
:1034D00060F48091E701882341F08150990B880FB7
:1034E000991F880F991FC80FD91F219623FF0EC05F
:1034F00061E0CE010E944A0A882309F46ECF612F51
:10350000CE010E947515181368CFD8CF60E0CE01A8
:103510000E944A0A882309F460CFCE010E948611D6
:10352000F2CFC43009F059CF80910E02682F70E0BD
:10353000762F66276627737090910F02692B6F5F55
:103540007F4F24E73AE0409110028C700E9498155A
:1035500044CF80E00E94290DE0910E02EF3F61F41C
:1035600080910F02811139CF80E090E0892B09F41E
:1035700034CF0E94000031CFE7FD0DC00091110251
:103580002091100240910F0270E060E08E2F90E0D9
:103590000E94061622CFE03C08F052C19091E00153
:1035A00097FF1BCF80910F02682F70E0EB01C09551
:1035B000D095CC0FDD1FCC0FDD1FC07CD170EF7319
:1035C000CE2B75956795262F2370B22E20910C0275
:1035D000253039F58C788C3021F50E9488118C17B4
:1035E0009D0721F0CF3FD14009F0F7CE80910F0227
:1035F00090E0982F882788279370C0911002C80FF9
:10360000D92FD11D21961091110261E0CE010E94A7
:103610004A0A612F882309F4E0CECE010E94751575
:10362000DCCE6E01A1E0CA1AD108CC0CDD1CCC0C9A
:10363000DD1CCB2886010F5F1F4F8091F801882386
:10364000F9F096FF41C0C80160E071E00E94452397
:10365000682F81E090E00E947515C80117FF02C035
:1036600081509F4F692F89E090E00E94751580E09E
:1036700090E0892B19F0C8010E9400001092F80117
:103680008091E00180FD39C080910C02843009F006
:103690004EC080910F028978813009F09ECE80E083
:1036A00090E0892B29F060911002C8010E9400006F
:1036B00080E090E0892B09F490CE409110026B2DB0
:1036C000C8010E94000089CEBE016F73772781E098
:1036D00090E00E947515BE0146E0759567954A9584
:1036E000E1F789E090E00E94751580E090E0892B79
:1036F00029F2CE010E940000C1CF86FF0CC00E94BB
:1037000088118017910709F4BFCF0D3FB7E01B0761
:103710000CF0BACF62CE0E9488118C179D0709F475
:10372000B3CFCF3FE1E0DE0709F4AECF56CE833012
:1037300069F540910F02F42FF170CF2E43FBDD2489
:10374000D0F880E090E0892B31F047702D2DBE013C
:10375000C8010E9400008091E00186FF0BC080E05C
:1037600090E0892B09F439CE4D2D6C2DC8010E94B3
:10377000000033CE80E090E0892B09F42ECE2D2D71
:103780004C2D6B2DCE010E94000027CE863009F013
:1037900024CE80910F02982F9978913021F08F7864
:1037A000803809F01ACE8091E00186FF25C00E9482
:1037B000881180179107E1F48091100290E0382F72
:1037C000222722273370C0911102C20FD32FD11D9F
:1037D00021961091120295958795959587958370FE
:1037E00099278230910589F0039709F40ECFF5CD22
:1037F0000D3F17400CF7F1CD0E9488118C179D07E3
:10380000D9F2CF3FD140C1F2E8CD14FFE6CD61E05F
:10381000CE010E944A0A882309F4DFCDCE010E941E
:103820008611912F977061E070E001C0660F9A9544
:10383000EAF713FF02C0682BF0CE60956823EDCE47
:10384000E83E08F0CACDE05CFF0B80910F020091CA
:103850001202209111024091100261E070E09E2F4F
:1038600097CE0E949E03685D7F4F8F4F9F4FF80158
:10387000668377838087918783E08583DF91CF910B
:103880001F910F91FF90EF90DF90CF90BF90089520
:103890001F920F920FB60F9211242F933F938F9385
:1038A0009F93AF93BF938091BC019091BD01A09174
:1038B000BE01B091BF013091BB0123E0230F2D3732
:1038C00058F50196A11DB11D2093BB018093BC0149
:1038D0009093BD01A093BE01B093BF018091C00140
:1038E0009091C101A091C201B091C3010196A11DA7
:1038F000B11D8093C0019093C101A093C201B09308
:10390000C301BF91AF919F918F913F912F910F90E4
:103910000FBE0F901F90189526E8230F0296A11D49
:10392000B11DD2CF1F920F920FB60F9211242F9379
:103930003F934F935F936F937F938F939F93AF9337
:10394000BF93EF93FF93E0910201F091030109957A
:10395000FF91EF91BF91AF919F918F917F916F9167
:103960005F914F913F912F910F900FBE0F901F903D
:1039700018951F920F920FB60F9211242F933F9319
:103980004F935F936F937F938F939F93AF93BF9367
:10399000EF93FF93E0910001F09101010995FF91F0
:1039A000EF91BF91AF919F918F917F916F915F91B7
:1039B0004F913F912F910F900FBE0F901F90189530
:1039C000CF93DF93CDB7DEB7FC018AA185FF14C08A
:1039D0002E89205C330B8F89922F978786878BA146
:1039E00080FF0DC02DA1205C330B8EA1922F918BF7
:1039F000808BDF91CF9108958E8190E0EECF8CA1E6
:103A000090E0F5CFCF93DF93CDB7DEB728E2FE018C
:103A10003596DF0101900D922A95E1F70C97DF9121
:103A2000CF910C94E01C6F70693011F481E008951F
:103A300080E008950A970C94131DE62FEF70E15073
:103A4000EA3018F5F0E0E95DF24E0C945923311D8F
:103A5000451D331D331D471D451D451D311D311DA0
:103A6000641D81E00895E0910A02F0910B029181BA
:103A7000842F8F71981748F0407EE091FC01F091FF
:103A8000FD0181E09081941710F580E020C0242F83
:103A9000207E30E085E0359527958A95E1F74F71D6
:103AA000E0910602F091070281E09285941708F4F4
:103AB00080E0E091FC01F091FD0191E0308132174E
:103AC00008F490E08923089581E04230F0F60895EB
:103AD0000A970C941D1D0895CF93DF9300D000D05A
:103AE00000D01F92CDB7DEB7789484B5826084BDD4
:103AF00084B5816084BD85B5826085BD85B58160F2
:103B000085BD80916E00816080936E00109281006F
:103B1000809181008260809381008091810081602A
:103B200080938100809180008160809380008091EB
:103B3000B10084608093B1008091B0008160809377
:103B4000B00080917A00846080937A0080917A003E
:103B5000826080937A0080917A00816080937A00FD
:103B600080917A00806880937A001092C10080E48E
:103B700080937C0080917A00806480937A008091A9
:103B80007A0086FDFCCF8091780060917900762FD5
:103B9000682F072E000C880B990B611571058105A4
:103BA000910511F00E94A32282E090E00E945F2321
:103BB0003C018FEA91E0D3018D939C9370920302B4
:103BC0006092020282E090E00E945F239A838983E0
:103BD00081EA91E0E981FA8191838083F093010287
:103BE000E093000286E190E00E945F237C0186E181
:103BF000D7011D928A95E9F7F70114828BE791E0CE
:103C00009183808383E991E0938782878BE991E0B8
:103C100095878487F0920502E09204028DE090E09F
:103C20000E945F236C01DC0115961C9290930702A1
:103C300080930602C3010E94B00CF601828790E0D7
:103C4000880F991F0E945F23D6011C969C938E9328
:103C50001B971B821C82B12CF6018285FB81F81711
:103C6000F0F4D301ED91FC910480F581E02D6B819E
:103C7000C3010995892B29F4B394EB81EF5FEB83A2
:103C8000EBCFD301ED91FC910280F381E02D6B81AC
:103C9000C3010995BC81B81780F78C83EECFFC81F6
:103CA000FF73AF2E81E0D6018C938EE090E00E94EE
:103CB0005F239D838C8389E691E0EC81FD81918374
:103CC000808386E08F01085F1F4FD801E82F1D9287
:103CD000EA95E9F79FEFAC81BD8119969C931997FE
:103CE0001296BC92129715969C9115979E7F1596E9
:103CF0009C93B89EC00111240E945F23EC81FD813A
:103D0000838394839C0190E0502F412FB91661F07A
:103D100086E0E52FF42FD90101900D928A95E1F705
:103D20009F5F2A5F3F4FF2CFAC81BD8116961C92F8
:103D3000169717961C921797F601B283A183AA20B3
:103D400009F479C18A2D90E0029663E070E00E9448
:103D50004523862E572E962E82E080838DE890E0B4
:103D60000E945F238C0187E591E0D80111969C9316
:103D70008E93F8013A96FD83EC8385E011928A9543
:103D8000E9F786E012968C93129713968C92A82CE2
:103D9000B52C82E1B82FBA9DC001BB9D900D1124B6
:103DA0000E945F23F801958384831086118690E03A
:103DB00080E040E055E02C812B833D813C83D8019D
:103DC0001496ED91FC911597E80FF91F2081216061
:103DD00020831496ED91FC911597E80FF91F11823D
:103DE0001496ED91FC91E80FF91F128230E020E06B
:103DF000F801A481B581A80FB91F529FB001539F4C
:103E0000700D1124A60FB71F1396EB81FC81652F4F
:103E100001900D926A95E1F72F5F3F4F23303105F6
:103E200039F74F5F4296491550F286E190E00E94C3
:103E30005F239D838C83DC0111961C921197189649
:103E40001C92FC011786108A118A128A1686138624
:103E500081E0848792E0958780834501880C991CD6
:103E60008A0C9B1C95828482C4010E945F23AC81D2
:103E7000BD811A969C938E931997009709F425C1DA
:103E8000A40170E060E00E949624EC81FD81B38281
:103E9000A28286E090E0EC81FD8197838683818118
:103EA000882341F061E086E00E941E0160E086E028
:103EB0000E94D200E1E1F1E0E491F0E0EE0FFF1F9B
:103EC000EF5FFE4F85919491AC81BD8154969C9398
:103ED0008E935397E3EFF0E0E4915596EC9355976A
:103EE000F801B783A68316968D919C9197FD0AC021
:103EF00061E00E941E0160E0AC81BD8116968C914C
:103F00000E94D20081E0EC81FD818183312C212C43
:103F1000512C412C0E94542224E030E040E050E03B
:103F20000E94C2224B015C01F4E08F0E911CA11C87
:103F3000B11C8B8224E130E0E1E0F0E041E0C80117
:103F4000820D931D9D838C83AC81BD81AE0FBF1FFD
:103F5000BF83AE83C901B4010E944523AE81BF81F6
:103F60001F966C9381E0840F31962C5E3F4FBB818E
:103F7000B81708F0B5C052E0B52EB40E0E94542216
:103F800022E030E040E050E00E94C22272E0972E32
:103F9000960EA12C2AE2249DF001259DF00D1124FE
:103FA000E00FF11FFD83EC830E94542222E030E0F9
:103FB00040E050E00E94C2226E5F2B2D30E0EC8189
:103FC000FD81E20FF31F178682E090E0220D331D82
:103FD000F901E80FF91FE00FF11F44E14687482F70
:103FE00001965FEF580F651798F7B40E0E945422A0
:103FF000EC81FD81EB0DF11D17868FEF808BB39463
:10400000B394A394A91480F2AC81BD811F96BC9295
:10401000BFEF4B1A5B0AEAE22E0E311CF3E04F169B
:10402000510409F077CFC8010E945C04D6011496B0
:104030001C930E9313971B82F6018285FB81F81760
:1040400008F079C0D301ED91FC910280F381E02D5D
:104050006B81C30109958C83D301ED91FC910480A0
:10406000F581E02D6B81C3010995BB80B394009766
:10407000C9F585E090E00E945F238C01FC0113826A
:10408000B4822C81208381818C7F8B7F81831282FB
:10409000E0910602F091070281819281DC01ED91AD
:1040A000FC910190F081E02D622F0995BB818B2F4F
:1040B00090E0880F991FF6010384F485E02DE80F46
:1040C000F91F11830083BB82B7CFAC81BD811596E8
:1040D0001C921E92149713961C921E921297D9CE80
:1040E000482F32CF019779F785E090E00E945F2357
:1040F0008C01DC0113961C9213971496BC921497B2
:10410000EC81EC9311968C91119781608D7F8B7F60
:1041100011968C93119712961C92E0910602F091E1
:10412000070283819481DC01ED91FC910190F08183
:10413000E02D6C81BACF89E190E00E945F23FC0101
:104140009C012E5F3F4F86E0D9011D928A95E9F7C9
:104150001186138689E491E091838083DD24DA94CB
:10416000D08A8FEF9FEF928B818B138A958B848BF4
:10417000168AF093FF01E093FE01168615862981C9
:104180003A81308F278B8CE0808785E08287A091F1
:104190000602B09107021A968C91848741E060E094
:1041A000CF010E9411170091FE011091FF01D8016B
:1041B0001A96CC9083E090E00E945F239A838983D3
:1041C0009093FD018093FC01FC01C0828C2D90E056
:1041D0000E945F23A981BA8112969C938E931197B6
:1041E00087E090E00E945F23FC0181E090E09183F2
:1041F000808393838283148215821682F09309024E
:10420000E0930802F801C08482E190E00E945F23FD
:104210009A838983DC011A961C921A971B961C922A
:104220001B971D96DC921D971E961C92FC0117860B
:10423000108A118A90930B0280930A02C0828DE14A
:1042400081838C2D880F828394859160948713825B
:1042500090E0880F991F0E945F23A981BA8114966C
:104260008C93149715969C93FC0190E080E0A981B3
:10427000BA8112962C912817190629F024F0119270
:1042800011920196F4CF83E0D82ECD9CC001112469
:104290000E945F23E981FA8197838683FDE0CF9EA8
:1042A000C00111240E945F23A981BA8119969C93B1
:1042B0008E9318971A961C921A971B961C92A70118
:1042C000445F5F4F60E0C8010E947012F894F09262
:1042D000FB01E092FA01F701D38261E083E00E94E2
:1042E0001E0160E0D70113968C910E94D20021E05C
:1042F000F70122831092F10182E08093F201EDE058
:10430000F1E0E491F0E0EE0FFF1FED51FF4F8591DA
:1043100094919093F4018093F301EFEEF0E0E49137
:10432000E093F50160E082E00E941E01EAECF1E01A
:1043300086E1DF011D928A95E9F782E990E090938A
:10434000C9018093C80182E590E09093C7018093F2
:10435000C6011092E001B1E0B093E1018FEF9FEF51
:104360009093F7018093F6011092F801D092C50165
:104370008091F5018093C40163E070E08091F101C8
:104380000E94AF008DE190E00E948611682F6F734C
:104390008DE190E00E9475158093F90160E087E05F
:1043A00090E00E94751560E088E090E00E9475152D
:1043B00080E00E94290DF7011282E0910A02F0913B
:1043C0000B0281E0D70150962D913C91232B09F4EB
:1043D00080E02485922F917020FD982F848590FB9A
:1043E00081F98487CF010E94EB07789480910402C1
:1043F00090910502DC01ED91FC910484F585E02D9E
:104400000995E0E0F0E0EF2B89F30E940000EECF89
:104410008F929F92AF92BF92CF92DF92EF92FF92D4
:10442000CF93DF93EC01688179818A819B8161154B
:1044300071058105910521F464E279ED8BE597E042
:104440002DE133EF41E050E00E94C22249015A01C0
:104450009B01AC01A7EAB1E40E94E1226B017C015F
:10446000ACEEB4EFA50194010E94EF22C60ED71E58
:10447000E81EF91EF7FE06C081E0C81AD108E1085F
:1044800080E8F80AC882D982EA82FB82C701B601B5
:104490009F77DF91CF91FF90EF90DF90CF90BF900B
:1044A000AF909F908F9008958F929F92AF92BF92FE
:1044B000CF92DF92EF92FF9260910401709105011B
:1044C00080910601909107016115710581059105A3
:1044D00021F464E279ED8BE597E02DE133EF41E0E3
:1044E00050E00E94C22249015A019B01AC01A7EA97
:1044F000B1E40E94E1226B017C01ACEEB4EFA501B6
:1045000094010E94EF22C60ED71EE81EF91EF7FE88
:1045100006C081E0C81AD108E10880E8F80AC09214
:104520000401D0920501E0920601F0920701C70153
:10453000B6019F77FF90EF90DF90CF90BF90AF9044
:104540009F908F900895609304017093050180936C
:104550000601909307010895F999FECF92BD81BDA0
:10456000F89A992780B50895262FF999FECF1FBA9A
:1045700092BD81BD20BD0FB6F894FA9AF99A0FBE8C
:1045800001960895052E97FB1EF400940E94D922EF
:1045900057FD07D00E94F42207FC03D04EF40C9480
:1045A000D92250954095309521953F4F4F4F5F4F01
:1045B000089590958095709561957F4F8F4F9F4F8F
:1045C00008950E941623A59F900DB49F900DA49F5F
:1045D000800D911D11240895B7FF0C94E1220E94D3
:1045E000E122821B930B0895A1E21A2EAA1BBB1B8A
:1045F000FD010DC0AA1FBB1FEE1FFF1FA217B307AF
:10460000E407F50720F0A21BB30BE40BF50B661FC4
:10461000771F881F991F1A9469F760957095809588
:1046200090959B01AC01BD01CF010895A29FB001FF
:10463000B39FC001A39F700D811D1124911DB29FD6
:10464000700D811D1124911D0895991B79E004C0FE
:10465000991F961708F0961B881F7A95C9F78095C1
:104660000895AA1BBB1B51E107C0AA1FBB1FA617B9
:10467000B70710F0A61BB70B881F991F5A95A9F70B
:1046800080959095BC01CD01089597FB072E16F4F7
:10469000009407D077FD09D00E94312307FC05D094
:1046A0003EF4909581959F4F0895709561957F4F49
:1046B0000895EE0FFF1F0590F491E02D09940F93DC
:1046C0001F93CF93DF938230910510F482E090E046
:1046D000E0911602F091170230E020E0B0E0A0E097
:1046E000309799F42115310509F44AC0281B390B7C
:1046F00024303105D8F58A819B816115710589F1D6
:10470000FB0193838283FE0111C0408151810281AC
:10471000138148175907E0F04817590799F4109783
:1047200061F012960C93129713961C933296CF0158
:10473000DF91CF911F910F9108950093160210936E
:104740001702F4CF2115310551F04217530738F005
:10475000A901DB019A01BD01DF01F801C1CFEF0121
:10476000F9CF9093170280931602CDCFFE01E20F8E
:10477000F31F819391932250310939832883D7CF36
:104780002091140230911502232B41F420910A014B
:1047900030910B01309315022093140220910801EF
:1047A000309109012115310541F42DB73EB74091F3
:1047B0000C0150910D01241B350BE0911402F09176
:1047C0001502E217F307A0F42E1B3F0B2817390739
:1047D00078F0AC014E5F5F4F2417350748F04E0F5D
:1047E0005F1F5093150240931402819391939FCFC2
:1047F000F0E0E0E09CCFCF93DF930097E9F0FC017D
:10480000329713821282A0911602B0911702ED0125
:1048100030E020E01097A1F420813181820F931FB6
:1048200020911402309115022817390709F061C050
:10483000F0931502E0931402DF91CF910895EA01FD
:10484000CE17DF07E8F54A815B819E0141155105CE
:10485000B1F7E901FB83EA8349915991C40FD51F50
:10486000EC17FD0761F4808191810296840F951FFA
:10487000E90199838883828193819B838A83F0E015
:10488000E0E012968D919C9113970097B9F52D91C8
:104890003C911197CD010296820F931F2091140233
:1048A000309115022817390739F6309751F51092D3
:1048B000170210921602B0931502A0931402BCCFF7
:1048C000D383C28340815181840F951FC817D907B4
:1048D00061F44E5F5F4F88819981480F591F518362
:1048E00040838A819B81938382832115310509F05E
:1048F000B0CFF0931702E09316029ECFFD01DC01CA
:10490000C0CF13821282D7CF81E090E0F8940C944C
:104910009D24FB01DC0104C08D910190801921F4DC
:1049200041505040C8F7881B990B0895DC0101C025
:0E4930006D9341505040E0F70895F894FFCF8A
:10493E00AA03AA030100000000001802800069000B
:10494E0001020305690007090B0D69000F1113150C
:10495E006900160000006A000406080A6A000C0EC0
:10496E0010126A00140000000005090D151D00014B
:10497E00020304050700000000B40AAA0A9D0A609B
:10498E00156A1900000000EA07E40516105C04AC75
:10499E0003380DAB0300000000A407CC072607E97F
:1049AE0007E0063206AB0300000000420C160CE8CE
:1049BE0018870B5D0BAB038F191D1D131DE01CF625
:1049CE00FF0000681D1A1DF4FF0000021D0000000C
:1049DE00009E0C9B0C6B0C650C5F0C00000000B075
:0649EE000CAA0CA10C0054
:00000001FF
